:100000000C94EC010C9409020C9409020C94090262
:100010000C9409020C9409020C9409020C94090234
:100020000C9409020C942D0C0C9409020C940902F6
:100030000C94FE140C9409020C9409020C9409020D
:100040000C9409020C9409020C94840B0C94090280
:100050000C945D040C9409020C94A5030C94090201
:100060000C94190D0C9409020C944B140C94090275
:100070000829573F9F2D49CBA5310F76C73493F2FE
:100080007E37D00D013AB60B613D2AAAAB3F000086
:10009000003F800000000A0A0D004E657574726111
:1000A0006C0048656164696E67486F6C64000A0D96
:1000B000537465756572756E673A20004F4B0A0D73
:1000C000000A0D4162676C65696368204C7566744F
:1000D000647275636B73656E736F722E2E000A0DFA
:1000E00042656E75747A6520506172616D657465E4
:1000F000727361747A202564000A0D496E69742E4A
:1001000020454550524F4D3A2047656E65726965EE
:1001100072652044656661756C742D506172616D05
:10012000657465722E2E2E000A0D3D3D3D3D3D3D10
:100130003D3D3D3D3D3D3D3D3D3D3D3D3D3D3D3DEF
:100140003D3D3D3D3D3D3D3D000A0D466C696768C6
:1001500074436F6E74726F6C205625642E25642074
:10016000002E0052616E67653A2533692D2533698B
:10017000005374656C6C756E673A202533690053C3
:100180006574706F696E7420202533690053657241
:10019000766F202000506F7469343A20202533692F
:1001A00000506F7469333A202025336900506F7412
:1001B00069323A202025336900506F7469313A2042
:1001C000202533690053746172743A202020202066
:1001D000253569004D657373776572743A20202563
:1001E0003569005269636874756E673A2020253559
:1001F00069004B6F6D7061737320202020202020D8
:1002000000456D70662E506567656C3A253569004E
:100210005370616E6E756E673A202025356900480F
:100220006F63682025346920282533692900526FBF
:100230006C6C20253469202825336929004E6963B8
:100240006B20253469202825336929004143432048
:100250002D2053656E736F720047696572202534D7
:100260006920282533692900526F6C6C2025346978
:10027000202825336929004E69636B2025346920C5
:100280002825336929004779726F202D2053656E28
:10029000736F720050333A25346920204B616EE44D
:1002A0006C65200050313A253469202050323A25BF
:1002B0003469200047733A253469202047693A257C
:1002C000346920004E693A2534692020526F3A255E
:1002D000346920004B373A25346920204B616EE4A5
:1002E0006C6520004B353A25346920204B363A2581
:1002F000346920004B333A25346920204B343A25A9
:10030000346920004B313A25346920204B323A259C
:10031000346920004B6F6D706173733A2020202583
:10032000356900526F6C6C3A202020202020253542
:1003300069004E69636B3A20202020202025356912
:1003400000616B742E204C6167650048F668656E2D
:10035000726567656C756E67004B65696E65200038
:100360004F66662020202020203A20253569004C49
:10037000756674647275636B3A2025356900536F36
:100380006C6C486F6568653A2025356900486F6573
:1003900068653A202020202025356900286329201F
:1003A000486F6C676572204275737300536574748F
:1003B000696E673A20256420005625642E25640066
:1003C0002B2B204D696B726F4B6F70746572202BF5
:1003D0002B005B25695D000011241FBECFEFD0E12B
:1003E000DEBFCDBF11E0A0E0B1E0E8E9F0E602C079
:1003F00005900D92AA38B107D9F716E0AAE8B1E046
:1004000001C01D92AB30B107E1F70E9440020C948D
:100410004B300C940000A2E0B0E00E943730802DF9
:1004200099270895FB01282F863008F025E0842FB6
:100430009927429FD0011124AC59BF4F019724F056
:1004400001900E943F30FACFA2E0B0E0022E0E945D
:100450003F300895CF93DF93FB01C42FDD27863013
:1004600008F085E0489FD0011124AC59BF4F219777
:1004700024F00E9437300192FACFDF91CF91089596
:100480000F931F93CF93DF9391E097B98FEF88B9C4
:100490008BE184B995B98EE38AB9579A87EF8BB906
:1004A00084B7877F84BF80916000886180936000FB
:1004B0001092600080ED97E09093A8018093A701CF
:1004C000109233021092320210929405109293050A
:1004D000109231021092300210922F0210922E02CE
:1004E00028980E94DA0C0E944C070E94E9140E948E
:1004F000130D0E943114789410924E048CE3809373
:100500004F0484E0809350048CE390E09F938F939A
:100510001F921F9289E491E09F938F931F920E94F4
:10052000E20888E291E09F938F931F920E94E20875
:10053000299AA1E0B0E00E943730802D2DB73EB758
:10054000265F3F4F0FB6F8943EBF0FBE2DBF8B33D3
:10055000A9F189EF90E09F938F931F920E94E20888
:100560000E94B41C4AE36BEB75E080E00E9412022B
:1005700001E00F900F900F90023049F40E94471C49
:100580004AE36BEB75E082E00E94120203E04AE36B
:100590006BEB75E0802F0E9412020F5F063060F354
:1005A00081E022E030E0D901082E0E943F308BE349
:1005B00021503040D901082E0E943F3002E010E067
:1005C000D8010E943730802D4AE36BEB75E00E9422
:1005D0002A02D8010E943730802D99279F938F934C
:1005E0008EED90E09F938F931F920E94E20880917E
:1005F000C3050F900F900F900F900F9080FF20C0B9
:1006000081EC90E09F938F931F920E94E20884EC0C
:1006100099E00E94180CEC010E943D100F900F9081
:100620000F90CE010E94210C8823D9F38CEB90E02F
:100630009F938F931F920E94E2080F900F900F904C
:100640000E946C1D289880ED97E09093A8018093FC
:10065000A70188EE93E0909349048093480485E5D0
:10066000809343048EEA90E09F938F931F920E94A1
:10067000E2088091C3050F900F900F9082FF03C096
:1006800082EA90E002C08AE990E09F938F931F92E4
:100690000E94E2080F900F900F9086E990E09F93E0
:1006A0008F931F920E94E2080E9464100F900F9097
:1006B0000F908091A401882379F11092A4010E94E7
:1006C0007D1E0E94251D289880910101882319F024
:1006D00081508093010180912D02882329F080911F
:1006E0002D02815080932D0220910401309105014B
:1006F0008091D30599272817390734F480ED97E0C6
:100700009093A8018093A7018091D201882319F4C6
:100710000E94311401C028980E9469070E94D707DF
:1007200080E090E00E94210C882319F2809134022D
:10073000882329F088B190E1892788B901C04498BD
:1007400084EF91E00E94180CB4CF1F920F920FB665
:100750000F9211248F939F93EF93FF938091000149
:100760008823E1F480919F019091A00101969093DC
:10077000A00180939F01FC01ED5FFC4FE081ED3013
:1007800019F08639910539F41092A00110929F0159
:1007900081E080930001E093C60004C01092A001A4
:1007A00010929F01FF91EF919F918F910F900FBE3B
:1007B0000F901F90189580912505813091F58091BB
:1007C000150590911605A0911705B0911805809315
:1007D000580590935905A0935A05B0935B058091F5
:1007E000190590911A05A0911B05B0911C058093E5
:1007F0005C0590935D05A0935E05B0935F058091C5
:100800001D0590911E05A0911F05B09120058093B4
:10081000600590936105A0936205B0936305109203
:10082000250580914204813031F480913604809313
:1008300070051092420480917204813091F580918C
:10084000620490916304A0916404B0916504809364
:10085000640590936505A0936605B0936705809144
:10086000660490916704A0916804B0916904809334
:10087000680590936905A0936A05B0936B05809114
:100880006A0490916B04A0916C04B0916D04809304
:100890006C0590936D05A0936E05B0936F05109253
:1008A000720480917005882339F0289A81E090E0E5
:1008B0009093D5028093D40208951F920F920FB6A1
:1008C0000F9211242F933F934F935F936F937F93D6
:1008D0008F939F93AF93BF93CF93DF93EF93FF9348
:1008E0008091C60080938E018091C00040918E015E
:1008F000887109F005C18091A101843009F48AC092
:10090000853050F48130D1F0813098F0823001F19F
:10091000833009F0F2C021C0863009F4ABC08630C4
:1009200008F48CC0873009F4D6C0883009F0E5C0DF
:10093000D8C0453B09F0E8C081E003C0423621F44D
:1009400082E08093A101E0C0453B09F4DDC0D5C041
:10095000413009F0D2C083E0F4CF409372054F5F7D
:1009600040930203809102038F5F8093310484E0FF
:100970008093A10180917205833031F0813161F162
:10098000813009F03FC014C082E394E090935D048D
:1009900080935C0423E535E0309300032093FF024D
:1009A000409690930A05809309058091420427C0E0
:1009B00081E195E090935D0480935C042AEC36E03D
:1009C000309300032093FF02449690930A0580938E
:1009D00009058091250513C08EE594E090935D0490
:1009E00080935C0427E136E0309300032093FF02FC
:1009F000449690930A058093090580917204809330
:100A0000730582C081E08093730510920A051092ED
:100A100009057AC0842F992790930C0580930B05C4
:100A200080910203840F809302038091310490919E
:100A30000203890F8093310485E083CF20910B0559
:100A400030910C05842F9927982F8827280F391F5C
:100A500030930C0520930B0580910203840F809343
:100A600002038091310490910203890F8093310435
:100A700086E067CF80910203840F80930203809108
:100A8000310490910203890F8093310480917305A2
:100A9000882381F4E0915C04F0915D048091FF0271
:100AA00090910003E817F90728F44193F0935D044F
:100AB000E0935C0480910B0590910C050197909355
:100AC0000C0580930B0580910B0590910C05892BEB
:100AD000D9F487E036CF80910203481771F488E09B
:100AE00030CF80913104481741F4E0910905F0912D
:100AF0000A05309711F081E080831092A10104C0B3
:100B00001092A1010E94DB030E94DB0340919A0135
:100B1000463910F01092990180918E018D3009F0C4
:100B20005CC080919901823009F057C01092990100
:100B3000A42FBB27FD01EF58FB4F3081ED01CE58AC
:100B4000DB4F288180919D0190919E01831B91092B
:100B5000821B91099F7090939E0180939D019C013F
:100B600096E0369527959A95E1F7235C20939C01B2
:100B7000982F9F73935C90939B018081281729F491
:100B80008881981711F491E006C0809191018F5FE0
:100B90008093910190E080918F01882309F064C0D7
:100BA000992309F461C081E080938F014093920101
:100BB000AD58BB4F8DE08C9380917504823509F060
:100BC00053C088E190E02CE00FB6F894A89580938C
:100BD00060000FBE2093600047C080919901813072
:100BE000D9F0813018F08230E9F530C080918E0163
:100BF000833239F480918F01882319F481E0809346
:100C0000990180918E018093730481E080939A0111
:100C100080918E01992715C082E080939901E42F7D
:100C2000FF2780918E01ED58FB4F80834F5F4093EB
:100C30009A0120918E0180919D0190919E01820FD9
:100C4000911D90939E0180939D010EC0E42FFF277C
:100C500080918E01ED58FB4F8083463938F3109216
:100C60009901E7CF10929901FF91EF91DF91CF9118
:100C7000BF91AF919F918F917F916F915F914F91B4
:100C80003F912F910F900FBE0F901F901895DC0190
:100C900020E030E040E050E0E3E0F3E005C0819187
:100CA000280F311D4F5F5F4F4A175B07C1F73F7039
:100CB000C90166E0969587956A95E1F7835CFD0129
:100CC000ED5FFC4F808311962F73235CFD01ED5F78
:100CD000FC4F2083AC5FBC4F8DE08C9310920001E1
:100CE000809103038093C6000895EF92FF920F93C3
:100CF0001F93CF93DF937A01722F93E290930303B4
:100D0000609304038093050303E010E060E0A6E035
:100D1000B3E046C0F701E60FF11D90816F5F71509F
:100D200019F4E0E040E00FC0F701E60FF11D40814B
:100D30006F5F715011F4E0E006C0F701E60FF11D9E
:100D4000E0816F5F7150892F86958695835C8C93C7
:100D50005527892F99278370907024E0880F991F59
:100D60002A95E1F79A0194E0369527959A95E1F74F
:100D7000822B835CED0189834F705070440F551FA7
:100D8000440F551F8E2F8295869586958370842BF0
:100D9000835C8A83EF73E35CEB830C5F1F4F1496D5
:100DA000772309F0B7CFC8010E944706DF91CF91A2
:100DB0001F910F91FF90EF9008950F931F93CF9382
:100DC000DF93EC01062F70E0A22FBB2712974AC0D9
:100DD000E42FFF27ED58FB4F30814F5FE42FFF27B3
:100DE000ED58FB4F50814F5FE42FFF27ED58FB4F2D
:100DF00010814F5FE42FFF27ED58FB4F20814F5F9D
:100E0000842F9927A817B90784F1701771F15D53E2
:100E1000FE01E70FF11D3D53330F330F852F8295F0
:100E20008F70382B3083613001F1912F9D537F5F9C
:100E3000FE01E70FF11D71505295507F892F869565
:100E40008695582B508363506F3F79F07E5FFE018B
:100E5000E70FF11D9295990F990F907C2D53922BCE
:100E600090837F5F662309F0B3CFDF91CF911F910D
:100E70000F9108951F93182F8A3019F48DE00E9466
:100E80003A078091C00085FFFCCF1093C60080E038
:100E900090E01F9108950895E1ECF0E088E18083EF
:100EA000A0ECB0E08C9182608C938081806880831C
:100EB0008081806480838AE28093C40088EC90E023
:100EC0000E94180C9093300480932F041092A1017B
:100ED000089580910001882309F468C080918A01F7
:100EE000882371F080910001882351F02BE043E4C6
:100EF00054E06091010387E40E94750610928A0114
:100F000080912F04909130040E94210C882321F4B9
:100F100080918C018823B1F080910001882391F0A9
:100F200022E346E255E06091010384E40E947506E5
:100F300010928C018AEF90E00E94180C909330047C
:100F400080932F0480918B018823F1F08091000120
:100F50008823D1F00E946D1010928B01809198012E
:100F60008F5F80939801843011F4109298018091E2
:100F7000980144E1849FA00111244A5E5E4F24E160
:100F800060E0805D0E94750680918D01882371F07C
:100F900080910001882351F02AE04EE454E06091F2
:100FA000010386E50E94750610928D0108951F9336
:100FB000CF93DF93CDB7DEB722970FB6F894DEBF9D
:100FC0000FBECDBF80918F01882309F498C08FEFA9
:100FD0008093010180917504813760F48C3608F0AC
:100FE0006FC0873609F440C08836F9F0833609F0BF
:100FF00084C008C0843759F1863791F1813709F0F0
:101000007CC036C02091920143E06BE083E494E021
:101010000E94DD068091C90190914504892B80933F
:10102000C90181E080938C0168C02091920143E066
:1010300062E0CE0101960E94DD068091C90199818E
:10104000892B8093C90181E080938B0156C0209148
:10105000920143E064E084E991E00E94DD064DC026
:1010600081E080938D0149C081E080938A0145C071
:101070002091920143E062E0CE0101960E94DD06DC
:1010800089818F3F89F0863010F085E089834AE3BB
:101090006BEB75E089810E942A0289812AE34BEB80
:1010A00055E06091010308C0109101030E940B02FA
:1010B0002AE34BEB55E0612F855B0E9475061DC04E
:1010C0002091920143E06AE38BEB95E00E94DD06FC
:1010D000809175044AE36BEB75E08B560E94120217
:1010E000809175048B56A2E0B0E0082E0E943F303C
:1010F0000E940B0299270E94681E10928F0122966F
:101100000FB6F894DEBF0FBECDBFDF91CF911F9118
:101110000895982F80917405813069F48091C801F9
:10112000E82FFF27EA5EFE4F90838F5F8093C80110
:1011300021E030E005C0892F0E943A07282F33278D
:10114000C90108951F93182F04C080E30E948908E5
:1011500011501116D4F31F9108951F93182F04C036
:1011600080E20E94890811501116D4F31F9108954E
:101170000F931F93CF93DF938C01EB0108C0F8010D
:101180000F5F1F4FE4918E2F0E94890821972097AF
:10119000B1F7DF91CF911F910F9108950F931F9396
:1011A000CF93DF938C01EB0106C0F80181918F0191
:1011B0000E94890821972097C1F7DF91CF911F9155
:1011C0000F9108952F923F924F925F926F927F926C
:1011D0008F929F92AF92BF92CF92DF92EF92FF9247
:1011E0000F931F93CF93DF93CDB7DEB7E3970FB67F
:1011F000F894DEBF0FBECDBF29968FAD299780939F
:101200007405CE01855B9F4F9D838C832B968EAD9D
:101210009FAD2B979FA78EA722243324210102C0C4
:10122000130124010EA51FA502C00F5F1F4FF80177
:10123000F490FF2019F0F5E2FF16B9F7B8018EA57A
:101240009FA5681B790B11F00E94B808FF2009F4D4
:1012500042C20F5F1F4F1FA70EA71982AC81BD812D
:101260001BAA1AAA9FEF99ABEEA5FFA5CF01019685
:101270009FA78EA7B49095E7B91621F08B2D8062B9
:10128000883789F4EBA9E0FF07C02D903D904D9081
:101290005C901397149607C08D919C9111971C0137
:1012A000442455241296F0E2BF1621F48981882344
:1012B000D9F685C083E2B81609F483C09AE2B9165C
:1012C00021F0EDE2BE1669F408C0FD011296E0813E
:1012D000EAABE7FFC9CFE195EAABFBA9F061FF7D7F
:1012E00072C08BE2B81609F46AC09EE2B916B1F575
:1012F0002EA53FA52F5F3F4FEEA5FFA584918A3213
:1013000021F0B82E20E030E01BC0FD011296408194
:10131000518157FF02C04FEF5FEF49AB3FA72EA7A8
:10132000A3CFC90103E0880F991F0A95E1F7220FA7
:10133000331F280F391F2B0D311D20533040B4901F
:1013400031968B2D80538A3060F3FFA7EEA7A90159
:1013500037FF02C04FEF5FEF49AB8DCFF0E3BF1611
:1013600031F48BA984FD80CF80628BAB7DCF8B2D38
:1013700081538930E8F420E030E0C901F3E0880FC0
:10138000991FFA95E1F7220F331F280F391F2B0DF4
:10139000311D20533040EEA5FFA5CF0101969FA738
:1013A0008EA7B4908B2D80538A3038F32AAB63CF4D
:1013B00098E6B91651F4EBA9E460EBAB55CFB982CE
:1013C00053CFFBA9F860FBAB4FCF8CE6B81621F4E6
:1013D0009BA991609BAB48CFBD83AC83E3E6BE166F
:1013E00039F41296BD83AC8312978C918E8318C109
:1013F000F4E4BF1639F084E6B81639F099E6B91668
:1014000059F503C0EBA9E160EBABFBA9F0FF08C005
:101410001496BD83AC835E904E903E902E900AC091
:101420001296BD83AC839E918E911C01442437FC9F
:101430004094542C57FC03C08AE088AB92C050946F
:10144000409430942094211C311C411C511C8DE28D
:1014500089839AE098AB85C0EFE4BE1629F0FFE6D9
:10146000BF1639F488E061C09BA991609BABE8E0AE
:1014700056C0F0E7BF1671F41296BD83AC839E91FF
:101480008E911C01442455248BA980648BAB78E792
:10149000B72E5EC0E3E7BE16D9F51296BD83AC83C6
:1014A000DE90CE90C114D10489F488E28E838EE65A
:1014B0008F8385E788878CE689878A8789E28B878F
:1014C0001C8666E0C62ED12CCC0EDD1EF9A9F7FDD8
:1014D00013C04F2F552747FD509560E070E0C601BF
:1014E0000E94702D009711F419A90DC08C1919A92B
:1014F00081174CF4182F07C0F60101900020E9F77E
:1015000031971E2F1C1919824201310140E094C00D
:1015100085E5B81631F095E7B91649F4EAE0E8AB8D
:101520001FC0FBA9F160FBAB8AE088AB19C098E54E
:10153000B91621F0E8E7BE1609F06EC0FBA9F3FD6D
:1015400002C080E1F2CF211431044104510419F4A6
:1015500090E198AB05C0EBA9E064EBABF0E1F8AB30
:10156000198289A987FD03C09BA99F7D9BAB21148C
:1015700031044104510461F4E9A9EE2349F46624DD
:10158000772443015EE2C52ED12CCC0EDD1E3EC079
:101590004EE2C42ED12CCC0EDD1EF8A9EF2EFF2476
:1015A00000271127C201B101A80197010E94FA2F5B
:1015B0006A3020F430E3A32EA60E08C027E5A22E41
:1015C000A60E88E5B81611F49FEDA922F601A292A5
:1015D0006F01C201B101A80197010E94FA2F3901E0
:1015E0004A012E143F044006510618F019012A0141
:1015F000D9CFF8A9F83051F48BA983FF07C090E345
:10160000A91621F080E3F60182936F01CE018C19B7
:10161000182F125D49A910C0BB2009F45CC0BE821E
:1016200019824201310100E096E0C92ED12CCC0E86
:10163000DD1E11E021E005C0212F042F011B07FD55
:1016400000E08981882319F0812F8F5F07C09BA953
:1016500096FD02C0812F02C0822F8E5FA82EA00EA1
:10166000EBA9EE2EFF2480E3482E512C4E205F2064
:101670004114510421F48AA98A190E94AD08898174
:10168000882329F061E070E0CE01019609C0E6FEF2
:1016900009C080E38A83BB8262E070E0CE010296DB
:1016A0000E94CE08F0E24F16510421F48AA98A194B
:1016B0000E94A208802F0E94A208612F772767FD51
:1016C0007095C6010E94CE08E4FEAACD8AA98A19A7
:1016D0000E94AD08A5CDE3960FB6F894DEBF0FBE0D
:1016E000CDBFDF91CF911F910F91FF90EF90DF90D1
:1016F000CF90BF90AF909F908F907F906F905F90B2
:101700004F903F902F9008951F920F920FB60F9217
:1017100011242F933F935F936F937F938F939F93A6
:10172000AF93BF938091AB0181508093AB018F3F0A
:1017300001F589E08093AB01809103018F5F817097
:1017400080930301882319F481E08093A4018091A0
:10175000A2019091A30101969093A3018093A2010D
:101760008091D201882329F08091D2018150809309
:10177000D2018091A7019091A801029758F0809121
:10178000A7019091A80101979093A8018093A701C8
:101790005A9A01C05A988091C30583FF3BC0349B7D
:1017A0000AC08091A5019091A60101969093A6018F
:1017B0008093A5012FC08091A5019091A601892B4E
:1017C00079F08091A5019091A601805A9F4040F444
:1017D0008091A5019091A60190931E0280931D0215
:1017E00080911D0290911E0220911F0230912002D3
:1017F000821B930B845E9D4F68E671E00E94E72F89
:10180000845B904090932202809321021092A60163
:101810001092A501BF91AF919F918F917F916F9190
:101820005F913F912F910F900FBE0F901F901895D1
:101830002091A2013091A3012F5F3F4F820F931F90
:1018400008952091A2013091A301821B930B892F4F
:10185000992786958074992708951F920F920FB645
:101860000F921124EF92FF920F931F932F933F93A8
:101870004F935F936F937F938F939F93AF93BF9398
:10188000CF93DF93EF93FF93809102018150809378
:1018900002018F3F09F073C083E88093B00080910C
:1018A0008901C82FDD27D093AA01C093A901809197
:1018B000E105E090DD0580FF1EC06091ED017091B3
:1018C000EE018091EF019091F001FF240027112794
:1018D00020E830E040E050E00E941C30C801B70131
:1018E0000E94B42F20E032E040E050E00E941C3023
:1018F000C20FD31F1DC06091ED017091EE01809168
:10190000EF019091F001FF240027112720E830E03B
:1019100040E050E00E941C30C801B7010E94B42F83
:1019200020E032E040E050E00E941C30C21BD30BAC
:10193000D093AA01C093A9012091A9013091AA01D5
:101940008091DE0599272817390734F08091DF054B
:1019500099278217930724F49093AA018093A901F1
:101960008091A9019091AA0190934D0580934C0517
:101970008093B3008091E0058093020104C083E06E
:101980008093B0005F98FF91EF91DF91CF91BF916D
:10199000AF919F918F917F916F915F914F913F9107
:1019A0002F911F910F91FF90EF900F900FBE0F900E
:1019B0001F9018958091A2019091A3010B9690938E
:1019C000AD018093AC0182E085BD83EA84BD17BC84
:1019D00088E788BD96E096BD83EC8093B000909335
:1019E000B100E0E7F0E0808182608083EEE6F0E025
:1019F0008081816080838AE08093B3001092B2007E
:101A000008952091A2013091A3012F5F3F4F280F2D
:101A1000391F8091A2019091A301A901481B590B84
:101A200057FFF7CF089510927C008FEE80937A00D5
:101A300008951F920F920FB60F921124EF92FF920A
:101A40000F931F932F933F934F935F936F937F93C6
:101A50008F939F93AF93BF93CF93DF93EF93FF93B6
:101A600010927A004091C4014F5F4093C4014150ED
:101A7000433009F41CC1443038F4413009F463C0E8
:101A8000423008F0B9C00DC0453009F450C14530AE
:101A900008F42AC1463009F46FC1473009F0CBC2BF
:101AA00052C22091D7013091D80180917800909155
:101AB0007900281B390B8091B2019091B301820FFC
:101AC000931F9093B3018093B2018091BC018F5F0B
:101AD0008093BC018091110290911202A091130297
:101AE000B0911402442737FD4095542F820F931F65
:101AF000A41FB51F8093110290931202A0931302AA
:101B0000B09314028091150290911602A0911702D1
:101B1000B0911802820F931FA41FB51F8093150266
:101B200090931602A0931702B093180281E080935D
:101B3000C5018091C2019091C30101969093C301A8
:101B40008093C2017CC2609178007091790080918D
:101B5000D5019091D601681B790B80910902909173
:101B60000A02A0910B02B0910C029B01442737FDA1
:101B70004095542F820F931FA41FB51F8093090215
:101B800090930A02A0930B02B0930C0280910D0275
:101B900090910E02A0910F02B0911002820F931F3C
:101BA000A41FB51F80930D0290930E02A0930F0205
:101BB000B093100280917800909179000A9710F408
:101BC00064E47DEF8091780090917900895E934084
:101BD00010F06CEB72E08091B0019091B101860F32
:101BE000971F9093B1018093B0018091BB018F5FEB
:101BF0008093BB0182E058C06091780070917900B9
:101C00008091D3019091D401681B790B80910102DE
:101C100090910202A0910302B09104029B0144271B
:101C200037FD4095542F820F931FA41FB51F80933B
:101C3000010290930202A0930302B09304028091E8
:101C4000050290910602A0910702B0910802820F4E
:101C5000931FA41FB51F8093050290930602A093C3
:101C60000702B093080280917800909179000A975A
:101C700010F464E47DEF8091780090917900895EA2
:101C8000934010F06CEB72E08091AE019091AF0147
:101C9000860F971F9093AF018093AE018091BA0198
:101CA0008F5F8093BA0184E08093C501C8C14091E1
:101CB00004015091050180917800909179009A017A
:101CC000220F331F240F351F63E070E00E94D32FD3
:101CD000260F371F369527953695279530930501A2
:101CE0002093040186E0E0CF8091DB019091DC013C
:101CF0002091780030917900821B930B90937605A8
:101D0000809375058091B4019091B501209175057E
:101D100030917605820F931F9093B5018093B401A3
:101D20008091BE018F5F8093BE0187E0BDCF80911F
:101D30007800909179002091D9013091DA01821BCD
:101D4000930B90937605809375058091B6019091E1
:101D5000B7012091750530917605820F931F9093FE
:101D6000B7018093B6018091BD018F5F8093BD0163
:101D70004093C50186E0E4C06091780070917900DD
:101D8000E090E701F090E8010091E9011091EA018B
:101D9000882777FD8095982F0E94292EA80197010A
:101DA0000E947D2D0E940C2E7093B9016093B801A2
:101DB0002091B8013091B901E0917505F091760557
:101DC000809180059091810597FF03C09095819542
:101DD0009F4F64E070E00E94E72FEB01CF01F7FF17
:101DE00003C0909581959F4F64E070E00E94E72FBB
:101DF000260F371F2C0F3D1F3093B9012093B801D8
:101E00008091B8019091B901029704F16091E701C6
:101E10007091E8018091E9019091EA0120E030E0C1
:101E200048E454E40E945F2E88230CF03CC060918B
:101E3000E7017091E8018091E9019091EA012AE0BF
:101E400037ED43EA5CE30E947E2D25C08091B80106
:101E50009091B9018F5F9F4F34F56091E7017091C8
:101E6000E8018091E9019091EA0120E030E046E14B
:101E700054E40E94622E1816B4F46091E701709148
:101E8000E8018091E9019091EA012AE037ED43EA07
:101E90005CE30E947D2D6093E7017093E8018093DD
:101EA000E9019093EA0181E08093BF01809178007D
:101EB000909179009093780580937705209119028D
:101EC00030911A0240911B0250911C028091B8017E
:101ED0009091B901AA2797FDA095BA2F280F391F15
:101EE0004A1F5B1F2093190230931A0240931B0272
:101EF00050931C02E0901902F0901A0200911B020C
:101F000010911C026091190270911A0280911B02BB
:101F100090911C0220E034E040E050E00E941C3030
:101F2000E21AF30A040B150BE0921902F0921A025E
:101F300000931B0210931C0283E08093C50187E08D
:101F40008093C4017CC08091850590918605209185
:101F5000780030917900820F931F909386058093CB
:101F6000850580917D058F5F80937D0580917D053E
:101F7000853008F460C0809178009091790090934A
:101F80000B0180930A0110927D0580917905909153
:101F90007A052091850530918605821B930B20914F
:101FA000350230913602821B930B9093C1018093CE
:101FB000C0016091850570918605E0900601F09062
:101FC00007010091080110910901882777FD80958C
:101FD000982FA8019701220F331F441F551F2E0D64
:101FE0003F1D401F511F620F731F841F951F24E068
:101FF00030E040E050E00E941C3020930601309316
:10200000070140930801509309012091790530910F
:102010007A058091060190910701A0910801B09185
:102020000901281B390B3093360220933502109298
:102030008605109285051092C5011092C401809109
:10204000C50180937C008FEE80937A00FF91EF9121
:10205000DF91CF91BF91AF919F918F917F916F91C0
:102060005F914F913F912F911F910F91FF90EF90B2
:102070000F900FBE0F901F901895CF93DF93C0E085
:10208000D0E0C7BD82E390E00E94010D81E691E0BF
:102090009F938F931F920E94E20880910A01909172
:1020A0000B010F900F900F908458934020F02196D1
:1020B000CA3FD10531F7C093820588EC90E00E94B9
:1020C000010DDF91CF910895E6E1F1E080E2819387
:1020D00091E0E636F907D9F70895FF920F931F9321
:1020E0008091C901282F3327C90181709070682F12
:1020F000882391F08091CA01882311F0815002C099
:10210000809166018093CA01E6E1F1E080E281936B
:1021100091E0E636F907D9F7A9014270507021FF26
:102120000DC08091CA018F5F8093CA01E6E1F1E0A2
:1021300080E2819391E0E636F907D9F7662321F032
:10214000452B11F01092CA0181E18093C801809162
:10215000CA0199279F938F9382ED93E09F938F936A
:10216000E1E0FE2EFF920E94E2080091CA010F906A
:102170000F900F900F900F90053009F4D7C10630E3
:1021800090F4023009F4B8C0033030F40023F1F0C9
:10219000013009F05BC34DC0033009F402C10430C3
:1021A00009F054C34BC1083009F498C2093038F41F
:1021B000063009F411C2073009F048C36CC2093077
:1021C00009F4C9C20A3009F041C303C31092C8011F
:1021D00080EC93E09F938F93FF920E94E20884E14A
:1021E0008093C8018CE390E09F938F931F921F927E
:1021F00089EB93E09F938F93FF920E94E20888E21D
:102200008093C8010E940B0299279F938F938CEAB9
:1022100093E09F938F93FF920E94E2088CE3809358
:10222000C8018CE993E09F938F93FF920E94E2088C
:102230008EC28091C30580FF47C01092C801809173
:102240003502909136029F938F938DE893E09F9390
:102250008F930F930E94E20884E18093C8018091DC
:102260003702909138029F938F938EE793E09F936C
:102270008F930F930E94E20888E28093C8018091B7
:102280000A0190910B019F938F938FE693E09F93A8
:102290008F930F930E94E2088CE38093C801809192
:1022A000820599279F938F9380E693E09F938F9366
:1022B0000F930E94E2088DB79EB744960FB6F8942C
:1022C0009EBF0FBE8DBFC7C284E18093C80189E560
:1022D00093E09F938F930F930E94E20888E280938C
:1022E000C8018BE493E09F938F930F930E94E208C1
:1022F0008DB79EB70696E2CF1092C80181E493E0B5
:102300009F938F93FF920E94E20884E18093C8011B
:102310006091ED017091EE018091EF019091F001DB
:1023200020E034E040E050E00E941C305F934F9387
:102330003F932F9382E393E09F938F93FF920E94AA
:10234000E20888E28093C8016091F5017091F6017E
:102350008091F7019091F80120E034E040E050E0F6
:102360000E941C305F934F933F932F9383E293E03F
:102370009F938F93FF920E94E2088CE38093C801A1
:1023800080911D0290911E029F938F9384E193E0B0
:102390009F938F93FF920E94E2088DB79EB7469657
:1023A0008DCF1092C8018091930590919405209152
:1023B0009105309192059F938F933F932F9384E0E3
:1023C00093E09F938F93FF920E94E20884E18093B1
:1023D000C8018091970590919805209195053091BD
:1023E00096059F938F933F932F9384EF92E09F9353
:1023F0008F93FF920E94E20888E28093C801809147
:102400009B0590919C052091990530919A059F9389
:102410008F933F932F9384EE92E09F938F93FF923D
:102420000E94E2088CE38093C80180919D05909101
:102430009E059F938F9384ED92E06FC01092C80128
:10244000E091BC05FF27EE0FFF1FE157FA4F2081F7
:102450003181E091BB05FF27EE0FFF1FE157FA4FD7
:10246000808191813F932F939F938F9384EC92E08F
:102470009F938F93FF920E94E20884E18093C801AA
:10248000E091BE05FF27EE0FFF1FE157FA4F2081B5
:102490003181E091BD05FF27EE0FFF1FE157FA4F95
:1024A000808191813F932F939F938F9384EB92E050
:1024B0009F938F93FF920E94E20888E28093C80165
:1024C000E091C005FF27EE0FFF1FE157FA4F208173
:1024D0003181E091BF05FF27EE0FFF1FE157FA4F53
:1024E000808191813F932F939F938F9384EA92E011
:1024F0009F938F93FF920E94E2088CE38093C80120
:10250000E091C105FF27EE0FFF1FE157FA4F8081D1
:1025100091819F938F9384E992E09F938F93FF9291
:102520000E94E2088DB79EB74A96C8CE1092C801A5
:1025300086E892E09F938F93FF920E94E20884E1E5
:102540008093C8012091D3013091D4018091AE01D4
:102550009091AF016091BA013F932F9377270E942A
:10256000E72F7F936F9387E792E09F938F93FF927C
:102570000E94E20888E28093C8012091D501309141
:10258000D6018091B0019091B1016091BB013F9360
:102590002F9377270E94E72F7F936F9388E692E02F
:1025A0009F938F93FF920E94E2088CE38093C8016F
:1025B0002091D7013091D8018091B2019091B3015F
:1025C0006091BC013F932F9377270E94E72F7F9361
:1025D0006F9389E592E056C01092C8018CE492E0B6
:1025E0009F938F93FF920E94E20884E18093C80139
:1025F0002091D9013091DA018091B6019091B70113
:102600006091BD013F932F9377270E94E72F7F931F
:102610006F938DE392E09F938F93FF920E94E20865
:1026200088E28093C8012091DB013091DC01809128
:10263000B4019091B5016091BE013F932F9377272C
:102640000E94E72F7F936F938EE292E09F938F9388
:10265000FF920E94E2088CE38093C8016091E70139
:102660007091E8018091E9019091EA01009177056C
:10267000109178050E940C2E7F936F931F930F93F8
:102680008FE192E09F938F93FF920E94E2088DB7B3
:102690009EB7489613CE84E18093C80180910401CF
:1026A000909105019F938F9380E192E09F938F9388
:1026B000FF920E94E20888E28093C80180912D0277
:1026C00099279F938F9381E092E09F938F93FF923E
:1026D0000E94E2088DB79EB70A96F0CD1092C8010D
:1026E00082EF91E09F938F93FF920E94E20884E132
:1026F0008093C80180912102909122029F938F9331
:1027000083EE91E09F938F93FF920E94E20888E20C
:102710008093C80180911D0290911E029F938F9318
:1027200084ED91E09F938F93FF920E94E2088CE3E7
:102730008093C80180911F02909120029F938F93F4
:1027400085EC91E09F938F93FF920E94E2088DB7F2
:102750009EB74296B3CD1092C80180912502909108
:1027600026029F938F9389EB91E09F938F93FF9223
:102770000E94E20884E18093C80180912702909131
:1027800028029F938F938DEA91E09F938F93FF92FE
:102790000E94E20888E28093C8018091290290910A
:1027A0002A029F938F9381EA91E09F938F93FF92E8
:1027B0000E94E2088CE38093C80180912B029091E3
:1027C0002C029F938F9385E991E09F938F93FF92C3
:1027D00070CD1092C8018DE891E09F938F93FF9286
:1027E0000E94E20884E18093C801809189019927C1
:1027F0009F938F938FE791E09F938F93FF920E9417
:10280000E20888E28093C8018091A9019091AA0111
:102810009F938F9381E791E09F938F93FF920E9404
:10282000E2088CE38093C8018091DF0599279F938C
:102830008F938091DE0599279F938F9383E691E094
:102840009F938F93FF920E94E20835CD0150009331
:1028500066011092CA011092C9011F910F91FF9059
:1028600008951092B9008AE28093B800089585EA2D
:102870008093BC0080E090E0089584E98093BC00E0
:1028800008951092B9008093BB0085E88093BC0046
:1028900080E090E008951F920F920FB60F921124DE
:1028A0008F939F93EF93FF938091CB018F5F8093E2
:1028B000CB018150833009F442C0843028F4813048
:1028C000A1F0823070F50CC0853009F448C0853025
:1028D000D8F1863009F44BC0873009F071C05BC075
:1028E0008091CC01880F8E5A14C08091CC018F5FEB
:1028F0008093CC018150813009F444C0813038F09C
:10290000823009F442C0833009F05AC041C080913E
:10291000C4021092B9008093BB0085E88093BC008C
:102920004FC084E98093BC008091CC01843018F4BE
:102930001092CB0102C01092CC0185EAEFCF8091BA
:10294000CD01880F8D5AE5CF8091CD018130D1F036
:102950008130E8F28230C9F0833091F519C080915E
:10296000BB00E091CD01FF27E957FA4F80838091AA
:10297000CD01813039F0813050F2823031F0833036
:10298000F9F406C08091C502C4CF8091D602C1CFB0
:102990008091EC02BECF8091CD019091BB00E82FD9
:1029A000FF27E957FA4F94838F5F8093CD018430DE
:1029B00010F01092CD0184E98093BC001092CB01FD
:1029C000FF91EF919F918F910F900FBE0F901F90ED
:1029D000189583EC80938100EFE6F0E080818062BF
:1029E00080831092D8011092D7011092D6011092D4
:1029F000D5011092D4011092D30108951F920F9225
:102A00000FB60F9211240F931F932F933F934F9361
:102A10005F936F937F938F939F93AF93BF93CF9366
:102A2000DF93EF93FF932091860030918700809190
:102A3000D0019091D101281B390B80918600909193
:102A400087009093D1018093D001C9018D5D95409D
:102A50008356994148F481E090E09093CF018093B0
:102A6000CE011092670154C0C091CE01D091CF0128
:102A7000CA30D1050CF04CC0C9018B5F9040845B1B
:102A8000914008F040C0A901425D5140FE01EE0FA7
:102A9000FF1FE157FA4F80819181FA01E81BF90B82
:102AA000CF01F7FF03C0909581959F4F06974CF497
:102AB00080912D02883C28F480912D02865F8093BE
:102AC0002D02FE01EE0FFF1F8F0101571A4FD80193
:102AD0002D913C91C901880F991F820F931F840F7C
:102AE000951F64E070E00E94E72FD8018D919C91C2
:102AF00011979B01281B390BEB55FA4F318320832B
:102B000011967C936E932196D093CF01C093CE0102
:102B1000FF91EF91DF91CF91BF91AF919F918F91F5
:102B20007F916F915F914F913F912F911F910F91E5
:102B30000F900FBE0F901F901895AF92BF92CF923B
:102B4000DF92EF92FF920F931F9310927A00809181
:102B5000BA01882369F08091AE019091AF01609134
:102B6000BA0177270E94E72F7093F8056093F70565
:102B70008091BB01882369F08091B0019091B101EF
:102B80006091BB0177270E94E72F7093F605609351
:102B9000F5058091BC01882369F08091B201909184
:102BA000B3016091BC0177270E94E72F7093040660
:102BB000609303068091BD018823D9F1E09000065F
:102BC000F09001066091B6017091B7012091BD01AE
:102BD0000027F7FC0095102F5701680143E0AA0C6D
:102BE000BB1CCC1CDD1C4A95D1F7AE18BF08C00A2F
:102BF000D10A882777FD8095982F34E0660F771FDC
:102C0000881F991F3A95D1F73327442755270E94EB
:102C10001C30A20EB31EC41ED51EC601B50128E08D
:102C200030E040E050E00E941C30309301062093D9
:102C300000068091BE018823D9F1E0900906F0904A
:102C40000A066091B4017091B5012091BE01002780
:102C5000F7FC0095102F5701680183E0AA0CBB1CFC
:102C6000CC1CDD1C8A95D1F7AE18BF08C00AD10A6A
:102C7000882777FD8095982FB4E0660F771F881F0F
:102C8000991FBA95D1F73327442755270E941C3046
:102C9000A20EB31EC41ED51EC601B50128E030E049
:102CA00040E050E00E941C3030930A062093090651
:102CB0008091BF018823A1F1E090FA05F090FB0517
:102CC0006091B8017091B9012091BF010027F7FC14
:102CD0000095102F57016801A3E0AA0CBB1CCC1C67
:102CE000DD1CAA95D1F7AE18BF08C00AD10A882703
:102CF00077FD8095982F3327442755270E941C3055
:102D0000A20EB31EC41ED51EC601B50128E030E0D8
:102D100040E050E00E941C303093FB052093FA0500
:102D20001092AF011092AE011092BA011092B1014F
:102D30001092B0011092BB011092B3011092B20137
:102D40001092BC011092B5011092B4011092BE0114
:102D50001092B7011092B6011092BD011092B90104
:102D60001092B8011092BF0180911102909112024D
:102D7000A0911302B09114028093FD019093FE0183
:102D8000A093FF01B0930002809101029091020292
:102D9000A0910302B09104028093ED019093EE01A3
:102DA000A093EF01B093F0018091090290910A0283
:102DB000A0910B02B0910C028093F5019093F60163
:102DC000A093F701B093F80180910502909106025B
:102DD000A0910702B09108028093F1019093F20153
:102DE000A093F301B093F40180910D0290910E0233
:102DF000A0910F02B09110028093F9019093FA0113
:102E0000A093FB01B093FC018FEE80937A00809138
:102E1000F7059091F805893C91057CF02091F70524
:102E20003091F8058091F7059091F805880F991F6A
:102E3000880F991F2052334015C08091F70590915B
:102E4000F80588539F4FA4F42091F7053091F805B9
:102E50008091F7059091F805880F991F880F991FA9
:102E6000205E3C4F820F931F9093F8058093F705E7
:102E70008091F5059091F605893C91057CF02091B3
:102E8000F5053091F6058091F5059091F605880FCE
:102E9000991F880F991F2052334015C08091F50566
:102EA0009091F60588539F4FA4F42091F505309139
:102EB000F6058091F5059091F605880F991F880F0A
:102EC000991F205E3C4F820F931F9093F6058093CD
:102ED000F50520912502309126028091BF05E82F4B
:102EE000FF27EE0FFF1FE157FA4F80819181825932
:102EF0009F4F281739071CF42F5F3F4F0CC080816C
:102F0000918182599F4F821793074CF42115310507
:102F100031F0215030403093260220932502209139
:102F20002702309128028091C005E82FFF27EE0F7D
:102F3000FF1FE157FA4F8081918182599F4F2817D7
:102F400039071CF42F5F3F4F0CC08081918182595B
:102F50009F4F821793074CF42115310531F0215012
:102F6000304030932802209327022091290230918B
:102F70002A028091C105E82FFF27EE0FFF1FE157BE
:102F8000FA4F8081918182599F4F281739071CF48D
:102F90002F5F3F4F0CC08081918182599F4F8217D4
:102FA00093074CF42115310531F021503040309316
:102FB0002A022093290220912B0230912C02809129
:102FC000C205E82FFF27EE0FFF1FE157FA4F808160
:102FD000918182599F4F281739071CF42F5F3F4F6B
:102FE0000CC08081918182599F4F821793074CF4C6
:102FF0002115310531F02150304030932C022093BF
:103000002B02809125029091260297FF05C0109215
:103010002602109225020AC08F3F910539F034F044
:103020008FEF90E0909326028093250280912702F3
:103030009091280297FF05C0109228021092270253
:103040000AC08F3F910539F034F08FEF90E09093F4
:103050002802809327028091290290912A0297FFEB
:1030600005C010922A02109229020AC08F3F9105D2
:1030700039F034F08FEF90E090932A028093290288
:1030800080912B0290912C0297FF05C010922C0288
:1030900010922B020AC08F3F910539F034F08FEF68
:1030A00090E090932C0280932B021F910F91FF9040
:1030B000EF90DF90CF90BF90AF90089510927A007C
:1030C0008091BA01882369F08091AE019091AF019F
:1030D0006091BA0177270E94E72F7093F8056093FB
:1030E000F7058091BB01882369F08091B001909130
:1030F000B1016091BB0177270E94E72F7093F6051D
:103100006093F5058091BC01882369F08091B2013C
:103110009091B3016091BC0177270E94E72F7093D3
:103120000406609303068091BD018823D1F060916D
:10313000B6017091B7012091BD01882777FD809578
:10314000982F34E0660F771F881F991F3A95D1F7A3
:103150003327442755270E941C30309301062093C3
:1031600000068091BE018823D1F06091B401709176
:10317000B5012091BE01882777FD8095982FB4E096
:10318000660F771F881F991FBA95D1F733274427F9
:1031900055270E941C3030930A062093090680911F
:1031A000BF01882399F06091B8017091B901209115
:1031B000BF01882777FD8095982F3327442755270F
:1031C0000E941C303093FB052093FA051092AF014A
:1031D0001092AE011092BA011092B1011092B0019A
:1031E0001092BB011092B3011092B2011092BC0177
:1031F0001092B5011092B4011092BE011092B70165
:103200001092B6011092BD011092B9011092B8014E
:103210001092BF018FEE80937A00209125023091A9
:1032200026028091BF05E82FFF27EE0FFF1FE15711
:10323000FA4F8081918182599F4F281739071CF4DA
:103240002F5F3F4F0CC08081918182599F4F821721
:1032500093074CF42115310531F021503040309363
:103260002602209325022091270230912802809186
:10327000C005E82FFF27EE0FFF1FE157FA4F8081AF
:10328000918182599F4F281739071CF42F5F3F4FB8
:103290000CC08081918182599F4F821793074CF413
:1032A0002115310531F02150304030932802209310
:1032B00027022091290230912A028091C105E82F2E
:1032C000FF27EE0FFF1FE157FA4F8081918182594E
:1032D0009F4F281739071CF42F5F3F4F0CC0808188
:1032E000918182599F4F821793074CF42115310524
:1032F00031F02150304030932A022093290220914E
:103300002B0230912C028091C205E82FFF27EE0F8F
:10331000FF1FE157FA4F8081918182599F4F2817F3
:1033200039071CF42F5F3F4F0CC080819181825977
:103330009F4F821793074CF42115310531F021502E
:10334000304030932C0220932B02809125029091E3
:10335000260297FF05C010922602109225020AC08D
:103360008F3F910539F034F08FEF90E09093260273
:1033700080932502809127029091280297FF05C033
:1033800010922802109227020AC08F3F910539F04F
:1033900034F08FEF90E09093280280932702809181
:1033A000290290912A0297FF05C010922A021092DA
:1033B00029020AC08F3F910539F034F08FEF90E079
:1033C00090932A028093290280912B0290912C02E3
:1033D00097FF05C010922C0210922B0208958F3F88
:1033E000910539F034F08FEF90E090932C028093A8
:1033F0002B0208951F938091C6058B3F98F08B3F59
:1034000019F4809125020EC08C3F19F48091270297
:1034100009C08D3F19F48091290204C08E3F21F428
:1034200080912B028093810180918101882319F47E
:103430001092810104C08F3F11F48093810180912B
:10344000C5058B3F98F08B3F19F4809125020EC083
:103450008C3F19F48091270209C08D3F19F48091A7
:10346000290204C08E3F21F480912B0280938001B9
:1034700080918001882319F41092800105C0843660
:1034800018F084E6809380018091C7058B3F98F007
:103490008B3F19F4809125020EC08C3F19F4809166
:1034A000270209C08D3F19F48091290204C08E3F84
:1034B00021F480912B0280938201809182018823E4
:1034C00019F41092820105C0843618F084E68093C6
:1034D00082018091C9058B3F98F08B3F19F4809150
:1034E00025020EC08C3F19F48091270209C08D3F40
:1034F00019F48091290204C08E3F21F480912B029F
:103500008093830180918301882319F410928301B1
:1035100004C08F3F11F4809383018091D0058B3FCD
:1035200098F08B3F19F4809125020EC08C3F19F45E
:103530008091270209C08D3F19F48091290204C0AF
:103540008E3F21F480912B0280938401809184012D
:10355000882319F41092840104C08F3F11F48093E2
:1035600084018091D1058B3F98F08B3F19F48091B5
:1035700025020EC08C3F19F48091270209C08D3FAF
:1035800019F48091290204C08E3F21F480912B020E
:1035900080938501809185018B3010F48AE002C010
:1035A0008F3F11F4809385018091D2058B3F98F075
:1035B0008B3F19F4809125020EC08C3F19F4809145
:1035C000270209C08D3F19F48091290204C08E3F63
:1035D00021F480912B0280938601809186018823BB
:1035E00019F41092860104C08F3F11F48093860174
:1035F0008091D7058B3F98F08B3F19F4809125027D
:103600000EC08C3F19F48091270209C08D3F19F438
:103610008091290204C08E3F21F480912B02809377
:10362000880180918801882319F41092880104C0D0
:103630008F3F11F4809388018091D8058B3F98F0DB
:103640008B3F19F4809125020EC08C3F19F48091B4
:10365000270209C08D3F19F48091290204C08E3FD2
:1036600021F480912B0280933902809139028823C2
:1036700019F41092390204C08F3F11F4809339027B
:103680008091D9058B3F98F08B3F19F480912502EA
:103690000EC08C3F19F48091270209C08D3F19F4A8
:1036A0008091290204C08E3F21F480912B028093E7
:1036B0003A0280913A02882319F410923A0204C027
:1036C0008F3F11F480933A028091DA058B3F98F096
:1036D0008B3F19F4809125020EC08C3F19F4809124
:1036E000270209C08D3F19F48091290204C08E3F42
:1036F00021F480912B0280933B0280913B0288232E
:1037000019F410923B0204C08F3F11F480933B02E6
:103710008091DB058B3F98F08B3F19F48091250257
:103720000EC08C3F19F48091270209C08D3F19F417
:103730008091290204C08E3F21F480912B02809356
:103740003C0280913C02882319F410923C0204C090
:103750008F3F11F480933C029091DC059B3FB0F0C9
:103760009B3F19F48091250204C09C3F29F480916D
:103770002702809389010CC09D3F19F48091290292
:10378000F8CF9E3F29F480912B02F3CF90938901CB
:1037900080918901882319F41092890104C08F3F18
:1037A00011F4809389019B3FB0F09B3F19F4809105
:1037B000250204C09C3F29F480912702809389014F
:1037C0000CC09D3F19F480912902F8CF9E3F29F447
:1037D00080912B02F3CF90938901809189018823F6
:1037E00019F41092890104C08F3F11F4809389016C
:1037F0009B3FB0F09B3F19F48091250204C09C3F91
:1038000029F480912702809389010CC09D3F19F40F
:1038100080912902F8CF9E3F29F480912B02F3CFAB
:103820009093890180918901882319F4109289016C
:1038300004C08F3F11F48093890110918801612F9A
:10384000772767FD7095872F972F0E94292E17FFE6
:1038500006C020E030E040E853E40E947E2D27E1DE
:1038600037EB41ED58E30E94502F60937C01709339
:103870007D0180937E0190937F018091CE0580939E
:1038800002068091CD058093F9051F91089581E08E
:103890008093BB0542E04093BC0583E08093BD0567
:1038A00024E02093BE0535E03093BF0586E0809389
:1038B000C00587E08093C1051092C3058EE1809317
:1038C000C4058BEF8093C6058AE08093C70592E319
:1038D0009093C5059093C9054093C8052093CA05E8
:1038E0001092CB0580E18093CC058FE08093CD05CD
:1038F0008AEF8093CE058AE18093CF0580E880939C
:10390000D0058FEA8093D1058093D2058AE5809314
:10391000D30583E28093D40584E18093D50510928A
:10392000D6053093D7051092D8051092D90510927C
:10393000DA051092DB0584E68093DC0588E280934B
:10394000DD051092E1059093DE0586E98093DF05A1
:103950003093E005A9EEB5E0E8E6F1E08CE00190F7
:103960000D928150E1F7089581E08093BB0552E00C
:103970005093BC0583E08093BD0544E04093BE05B1
:1039800035E03093BF0586E08093C00587E08093E3
:10399000C10528E02093C2051092C3059EE19093D3
:1039A000C4058BEF8093C6058AE08093C70586E443
:1039B0008093C5059093C9055093C8054093CA05E7
:1039C0002093CB0580E18093CC058FE08093CD05DB
:1039D0008AEF8093CE058AE18093CF0580E88093BB
:1039E000D00588E78093D10596E99093D2058AE5C2
:1039F0008093D30583E28093D40584E18093D50539
:103A00001092D6053093D7051092D8051092D9059B
:103A10001092DA051092DB0584E68093DC0588E2DB
:103A20008093DD051092E10582E38093DE0590939B
:103A3000DF053093E005A9EEB5E0E0E7F1E08CE0CA
:103A400001900D928150E1F708958091340288230E
:103A500001F51092C5021092C4021092D602109283
:103A6000EC0280919401882311F08093C40280912C
:103A70009501882311F08093C502809196018823D7
:103A800011F08093EC0280919701882311F08093CC
:103A9000D6028091C40299279093510580935005D6
:103AA0008091C50299279093530580935205809188
:103AB000EC02992790935505809354058091D60286
:103AC000992790935705809356051092CB01109239
:103AD000CC010E9437140895CF93DF931092DA013E
:103AE0001092D9011092DC011092DB0180E090E08D
:103AF000A0E0B0E08093E7019093E801A093E90192
:103B0000B093EA011092D4011092D3011092D60121
:103B10001092D5011092D8011092D7010E945E1820
:103B200085E090E00E94180CEC01CE010E94210C6F
:103B30008823D9F30E945E188091C30580FF10C0CE
:103B400080910A0190910B01875B934038F480913A
:103B50000A0190910B018E5E924010F40E943D107C
:103B60008091F7059091F80597FF03C09095819596
:103B70009F4F9093D4018093D3018091F50590914C
:103B8000F60597FF03C0909581959F4F9093D601BE
:103B90008093D501809103069091040697FF03C09E
:103BA000909581959F4F9093D8018093D7018091F4
:103BB000090690910A0697FF03C0909581959F4F43
:103BC00060E170E00E94E72F7093DC016093DB01FD
:103BD000809100069091010697FF03C09095819512
:103BE0009F4F60E170E00E94E72F7093DA016093CD
:103BF000D9016091770570917805882777FD8095C8
:103C0000982F0E94292E6093E7017093E80180931A
:103C1000E9019093EA0110920102109202021092BF
:103C200003021092040210920502109206021092F2
:103C30000702109208021092090210920A021092D2
:103C40000B0210920C0210920D0210920E021092B2
:103C50000F02109210021092110210921202109292
:103C60001302109214021092F8051092F7051092A8
:103C7000F6051092F5051092040610920306809145
:103C8000060190910701A0910801B091090190935C
:103C90007A05809379051092C1011092C0011092AB
:103CA000190210921A0210921B0210921C028091AB
:103CB0001D0290911E029093200280931F0282E3C6
:103CC00090E09093A8018093A701DF91CF91089590
:103CD0001F93182F0EC080913402882361F484E66C
:103CE00090E09093A8018093A7018AEF90E00E9452
:103CF000010D115080F71F9108952F923F924F921E
:103D00005F926F927F928F929F92AF92BF92CF926B
:103D1000DF92EF92FF920F931F93CF93DF93CDB774
:103D2000DEB724970FB6F894DEBF0FBECDBF0E945A
:103D30009D15299AE091BD05AE2FBB27AA0FBB1F89
:103D4000A157BA4F0D90BC91A02D9D0128583F4F0F
:103D50003A83298337FF02C01A82198280912D028B
:103D6000843608F04AC080910101882331F484EF41
:103D700091E09093A8018093A701809148029091CF
:103D80004902009731F001979093490280934802CD
:103D900004C01092340210922302289A80914302A8
:103DA00090914402815D974028F18091D405482F7D
:103DB00055275A83498381E080932302E091BB0514
:103DC000FF27EE0FFF1FE157FA4F11821082E0919B
:103DD000BC05FF27EE0FFF1FE157FA4F118210823B
:103DE000E091BE05FF27EE0FFF1FE157FA4F11824A
:103DF0001082CEC110923402CBC180912D028D3839
:103E000008F4C6C1109223028091D50522E3829F57
:103E1000C0011124909349028093480269817A81FC
:103E2000693271056CF080914302909144027FEFFA
:103E30008F3F970781F1019690934402809343024C
:103E40008091430290914402883C910520F0898141
:103E50009A81889704F510925E0210925F02109288
:103E600060021092610210925A0210925B0210924C
:103E70005C0210925D0210921102109212021092D6
:103E80001302109214021092150210921602109250
:103E9000170210921802E981FA81E93CF1050CF44D
:103EA000D6C080913402882309F072C1E091BE052A
:103EB000FF27EE0FFF1FE157FA4F808191818C346D
:103EC00091050CF4C1C0809147028F5F8093470237
:103ED000893C08F45DC129980E946C1D109234023F
:103EE0001092470210924402109243028091BB0547
:103EF000282F3327F901EE0FFF1FE157FA4F80817A
:103F00009181873491059CF4E091BC05FF27EE0F69
:103F1000FF1FE157FA4F0190F081E02DF7FF03C03A
:103F2000F095E195FF4FE734F1050CF46CC08091FA
:103F3000BC05682F7727DB01AA0FBB1FA157BA4F1B
:103F40008D919C911197873491053CF0F901EE0F0A
:103F5000FF1FE157FA4F808191818D919C918734A9
:103F6000910564F0F901EE0FFF1FE157FA4F8081D0
:103F700091818734910514F042E001C041E0FB01DA
:103F8000EE0FFF1FE157FA4F808191818634910532
:103F90005CF4F901EE0FFF1FE157FA4F8081918128
:103FA000873491050CF043E0FB01EE0FFF1FE15752
:103FB000FA4F808191818A5B9F4F5CF4F901EE0F8B
:103FC000FF1FE157FA4F80819181873491050CF0F2
:103FD00044E0660F771F61577A4FFB018081918122
:103FE0008A5B9F4F5CF4220F331F21573A4FF90130
:103FF00080819181863491050CF445E0A2E0B0E027
:10400000042E0E943F300E940B024AE36BEB75E0E6
:104010000E942A020E940B020E94681E8091C30522
:1040200080FFB6C080910A0190910B01875B93409D
:1040300040F480910A0190910B018E5E924008F04D
:10404000A7C00E943D10A4C010924702A1C04981A0
:104050005A81433251050CF09BC08091BE05482F18
:104060005527FA01EE0FFF1FE157FA4F808191812A
:10407000855B9F4F0CF06DC0809146028F5F8093EF
:104080004602893C08F467C088EC8093460281E0D0
:1040900090E0909344028093430281E08093340245
:1040A0001092560210925702109258021092590222
:1040B0001092110210921202109213021092140226
:1040C0001092150210921602109217021092180206
:1040D0001092010210920202109203021092040246
:1040E0001092090210920A0210920B0210920C0216
:1040F0008091ED019091EE01A091EF01B091F0015E
:104100008093050290930602A0930702B0930802E1
:104110008091F5019091F601A091F701B091F8011D
:1041200080930D0290930E02A0930F02B0931002A1
:1041300010925E0210925F02109260021092610271
:1041400010925A0210925B0210925C0210925D0271
:1041500002C010924602440F551F41575A4FFA01B0
:10416000808191818C3491058CF0809145028F5F24
:1041700080934502893C60F01092340288EC809371
:104180004502109244021092430202C0109245026E
:1041900080916701815080936701809167018F3F13
:1041A00029F080912302882309F412C10E94FA1990
:1041B000E091BB05FF27EE0FFF1FDF01A157BA4FAC
:1041C0008D919C916091CA057727EB55FA4F20811C
:1041D00031814091CB055527FC01E69FC001E79F47
:1041E000900DF69F900D1124F901E49F9001E59F39
:1041F000300DF49F300D1124820F931F90932F02E6
:1042000080932E02E091BC05FF27EE0FFF1FDF0118
:10421000A157BA4F8D919C91EB55FA4F2081318176
:10422000FC01E69FC001E79F900DF69F900D1124C1
:10423000B901649F9001659F300D749F300D11246A
:10424000820F931F9093310280933002E091BE055C
:10425000FF27EE0FFF1FE157FA4F80819181909564
:1042600081959F4F90933302809332021091850184
:10427000612F772767FD7095872F972F0E94292E32
:1042800017FF06C020E030E040E853E40E947E2D96
:1042900020E030E040E251E40E947E2D20E030E05A
:1042A00040E85BE30E94502F5B016C0160930506C0
:1042B0007093060680930706909308061091860176
:1042C000612F772767FD7095872F972F0E94292EE2
:1042D00017FF06C020E030E040E853E40E947E2D46
:1042E00020E030EE4BE257E40E94C62D6093FC05BF
:1042F0007093FD058093FE059093FF058091C305A3
:1043000082FF0CC080E090E0A0E0B0E08093FC056C
:104310009093FD05A093FE05B093FF0520E030E0EB
:1043200040E050E0C601B5010E945F2E882364F48E
:1043300080E090E0A0E0B0E0809305069093060650
:10434000A0930706B093080620E030E040E050E07C
:104350006091FC057091FD058091FE059091FF052F
:104360000E945F2E882364F480E090E0A0E0B0E03B
:104370008093FC059093FD05A093FE05B093FF0587
:1043800080912302882321F110923302109232028D
:1043900010922F0210922E021092310210923002CF
:1043A0008DEC9CECACECBDE3809305069093060687
:1043B000A0930706B09308068AE097EDA3EABBE353
:1043C0008093FC059093FD05A093FE05B093FF0537
:1043D0008091C2019091C3018D54914008F4BCC0FA
:1043E0002091F1013091F2014091F3015091F401DB
:1043F0008091ED019091EE01A091EF01B091F0015B
:10440000B901681B790B70934D0260934C022091A7
:10441000F9013091FA014091FB015091FC0180912A
:10442000F5019091F601A091F701B091F801281BD8
:10443000390B30934B0220934A021092C301109221
:10444000C201673A710534F08091D3019091D40193
:10445000019608C06A557F4F4CF48091D30190912A
:10446000D40101979093D4018093D301273A310569
:1044700034F08091D5019091D601019608C02A555B
:104480003F4F4CF48091D5019091D60101979093C4
:10449000D6018093D5018091150290911602A091CA
:1044A0001702B0911802873A9105A105B1054CF0A9
:1044B0008091D7019091D80101979093D801809372
:1044C000D7018091150290911602A0911702B09128
:1044D00018028A559F4FAF4FBF4F4CF48091D701C0
:1044E0009091D80101969093D8018093D7011092B2
:1044F0007A008091ED019091EE01A091EF01B091D1
:10450000F0018093050290930602A0930702B093F6
:1045100008028091F5019091F601A091F701B09108
:10452000F80180930D0290930E02A0930F02B093B6
:1045300010028091FD019091FE01A091FF01B091C8
:1045400000028093150290931602A0931702B09375
:1045500018028FEE80937A006091ED017091EE0168
:104560008091EF019091F001A090CF05BB24CC2465
:10457000DD24E0900006F0900106A60195010E945E
:104580001C300027F7FC0095102F2E193F09400B17
:10459000510BCA01B90120E130E040E050E00E9437
:1045A0001C3039014A012093520230935302409348
:1045B0005402509355026091F5017091F60180917B
:1045C000F7019091F801E0900906F0900A06A60123
:1045D00095010E941C300027F7FC0095102F2E1922
:1045E0003F09400B510BCA01B90120E130E040E026
:1045F00050E00E941C3020934E0230934F024093B3
:10460000500250935102F5EF6F16F1E07F06F0E093
:104610008F06F0E09F062CF084EF91E0A0E0B0E080
:104620000DC06CE066166EEF76066FEF86066FEFD4
:10463000960664F48CE09EEFAFEFBFEF80935202DA
:1046400090935302A0935402B0935502253F71E01A
:10465000370770E0470770E057072CF084EF91E0D0
:10466000A0E0B0E009C02C503E4F4F4F5F4F64F4C4
:104670008CE09EEFAFEFBFEF80934E0290934F021E
:10468000A0935002B093510210927A0080910102DF
:1046900090910202A0910302B09104022091520273
:1046A000309153024091540250915502821B930B5A
:1046B000A40BB50B8093010290930202A093030216
:1046C000B09304028091090290910A02A0910B021A
:1046D000B0910C0220914E0230914F024091500255
:1046E00050915102821B930BA40BB50B80930902CE
:1046F00090930A02A0930B02B0930C0280913202B5
:10470000909133025C01CC24B7FCC094DC2CA092C5
:104710005602B0925702C0925802D092590297FFA7
:1047200003C0909581959F4F84973CF08091C3057D
:1047300084FD03C081E080933F026090110270907D
:1047400012028090130290901402C501B7FE03C0BC
:10475000909581959F4F7C010027F7FC0095102FC5
:104760002091CC05332744275527C601B5010E9467
:10477000B42F9B01AC01C801B7010E94B42F20E007
:1047800031E040E050E00E941C30442737FD409566
:10479000542F621A730A840A950A60921102709269
:1047A0001202809213029092140280911102909151
:1047B0001202A0911302B091140281539547A040B8
:1047C000B04064F080E395E7A0E0B0E08093110290
:1047D00090931202A0931302B093140280911102DD
:1047E00090911202A0911302B0911402805D9A4838
:1047F000AF4FBF4F64F480ED9AE8AFEFBFEF809307
:10480000110290931202A0931302B09314028FEE40
:1048100080937A0080911D0290911E02892B09F4E9
:10482000A1C08091C30583FF9DC06091ED0170918F
:10483000EE018091EF019091F00120E032E040E044
:1048400050E00E941C30890137FF03C0109501958C
:104850001F4F6091F5017091F6018091F7019091E1
:10486000F80120E032E040E050E00E941C30B90145
:1048700037FF03C0709561957F4F601771070CF487
:10488000B80169317105A4F480913F02882381F059
:1048900080913D0290913E02892B51F480911D023E
:1048A00090911E029093200280931F0210923F026B
:1048B000209184013327629FC001639F900D729FF6
:1048C000900D112460E470E00E94E72FA901461BBF
:1048D000570B141615060CF03FC010927A00209169
:1048E0003D0230913E022115310561F50091110222
:1048F0001091120220911302309114028091210232
:1049000090912202BC01649FC001659F900D749F2D
:10491000900D112460E270E00E94E72F882777FD58
:104920008095982F060F171F281F391F009311021B
:104930001093120220931302309314028FEE80938F
:104940007A0010C08FEE80937A002150304030936F
:104950003E0220933D0206C084EF91E090933E0218
:1049600080933D028091390299279093E7028093CA
:10497000E60280913A0299279093E9028093E80237
:1049800080913B0299279093E3028093E202809109
:104990003C0299279093E5028093E40289E190E03C
:1049A0009093D3028093D2028091250290912602A7
:1049B0001816190614F40E94792980912502909105
:1049C0002602892B71F485E090E09093DD028093BC
:1049D000DC021092BF021092BE021092C10210922D
:1049E000C002809137058F5F809337058091400228
:1049F0008150809340028F3F09F078C081E380931B
:104A000040026091ED017091EE018091EF01909173
:104A1000F001E090CF05FF2400271127A80197019E
:104A20000E941C3030933905209338056091F501C0
:104A30007091F6018091F7019091F801A80197011A
:104A40000E941C3030933B0520933A05809100066C
:104A50009091010690933D0580933C058091090655
:104A600090910A0690933F0580933E05809103063E
:104A70009091040690934105809340058091350202
:104A800090913602909343058093420560911902FC
:104A900070911A0280911B0290911C0220E032E07A
:104AA00040E050E00E941C303093450520934405BF
:104AB00089819A81909347058093460580911D02D4
:104AC00090911E02909349058093480580911D02A4
:104AD00090911E0290934B0580934A0580911D0290
:104AE00090911E0290934D0580934C056091ED01CD
:104AF0007091EE018091EF019091F0012090FC0502
:104B00003090FD054090FE055090FF05E090F705C0
:104B1000F090F805609005067090060680900706F4
:104B2000909008060E94292EA20191010E94502F08
:104B30005B016C010027F7FC0095102FC801B7013D
:104B40000E94292EA40193010E94502F9B01AC01C9
:104B5000C601B5010E947E2D0E940C2E7093F805AF
:104B60006093F7056091F5017091F6018091F7016E
:104B70009091F801E090F505F090F6050E94292E3D
:104B8000A20191010E94502F5B016C010027F7FCEC
:104B90000095102FC801B7010E94292EA40193018E
:104BA0000E94502F9B01AC01C601B5010E947E2DD1
:104BB0000E940C2E7093F6056093F5056091030634
:104BC00070910406A090FD01B090FE01C090FF011D
:104BD000D0900002882777FD8095982F0E94292E7B
:104BE0007B018C0120E030E040E05FE3C401B301D1
:104BF0000E94502F9B01AC01C801B7010E94502FA9
:104C00007B018C01C601B5010E94292EA2019101F0
:104C10000E94502F9B01AC01C801B7010E947E2D5C
:104C20000E940C2E70930406609303068091F70592
:104C30009091F8058150984034F080E098E090938E
:104C4000F8058093F7058091F7059091F80580505D
:104C5000984F34F480E098EF9093F8058093F7052F
:104C60008091F5059091F6058150984034F080E0F0
:104C700098E09093F6058093F5058091F505909165
:104C8000F6058050984F34F480E098EF9093F60545
:104C90008093F50580910306909104068150984019
:104CA00034F080E098E090930406809303068091AE
:104CB0000306909104068050984F34F480E098EFFA
:104CC00090930406809303068091C305992780FF83
:104CD000CDC02091810181FF0EC02233B0F48091BC
:104CE00035029091360244979093380280933702B0
:104CF000109224020DC08091C805289FC001112484
:104D00004497909338028093370281E08093240285
:104D100080912302882321F01092380210923702EA
:104D2000209135023091360240913702509138027D
:104D3000421753070CF09AC080912402882309F48B
:104D400095C0241B350B809182019927BC01269FB9
:104D5000C001279F900D369F900D112460E170E0F7
:104D60000E94E72F09811A81061B170B2091C001B1
:104D70003091C101809180019927FC012E9FC001D3
:104D80002F9F900D3E9F900D112468E070E00E94CF
:104D9000E72F061B170B6091190270911A02809180
:104DA0001B0290911C0220E032E040E050E00E94A3
:104DB0001C30CA01B90120918301332744275527AC
:104DC0000E94B42F20E230E040E050E00E941C300E
:104DD000FFEF2E3C3F0714F42EEC3FEF8091410291
:104DE00090914202AC0174E0440F551F7A95E1F7AF
:104DF000481B590B2333310514F022E330E0021B2A
:104E0000130BCA01800F911F60E170E00E94E72F31
:104E100070934202609341028091C40599276817FC
:104E200079078CF429813A81281739072CF090935F
:104E300042028093410207C049815A815093420245
:104E4000409341020DC080914102909142026981DC
:104E50007A816817790724F47093420260934102C3
:104E600080914102909142029A838983C090030607
:104E7000D09004068091560290915702C81AD90A20
:104E800095E6C916D10424F064E6C62ED12C09C0DB
:104E9000ECE9CE16EFEFDE0624F45CE9C52E5FEFF9
:104EA000D52E409078015090790160907A017090F1
:104EB0007B016091F7057091F80520912E023091E9
:104EC0002F024091BE025091BF02241B350B621B82
:104ED000730B882777FD8095982F0E94292E9B01C0
:104EE000AC01C301B2010E94502F0E940C2E70939E
:104EF000D1026093D0028091D0029091D1028C01B6
:104F0000222717FD2095322F80915E0290915F023B
:104F1000A0916002B0916102080F191F2A1F3B1F68
:104F200000935E0210935F0220936002309361024F
:104F30001016110612061306ACF4C80117FF03C0C1
:104F4000909581959F4F60E071E00E94E72F6F5F21
:104F50007F4F882777FD8095982F061B170B280B0E
:104F6000390B14C0C80117FF03C0909581959F4F5E
:104F700060E071E00E94E72F6F5F7F4F882777FD29
:104F80008095982F060F171F281F391F00935E0268
:104F900010935F02209360023093610280915E0261
:104FA00090915F02A0916002B09161028138FEE3AE
:104FB0009F07F0E0AF07F0E0BF072CF080E89EE32A
:104FC000A0E0B0E009C08058914CAF4FBF4F64F4EF
:104FD00080E891ECAFEFBFEF80935E0290935F02A9
:104FE000A0936002B09361026091D0027091D102EF
:104FF00080907C0190907D01A0907E01B0907F0117
:10500000882777FD8095982F0E94292E7B018C019F
:1050100060915E0270915F028091600290916102E6
:105020000E94292E9B01AC01C501B4010E94502FA2
:105030009B01AC01C801B7010E947E2D0E940C2E7D
:105040009601260F371F49815A81240F351F2224CC
:105050004A30510514F441E0242E37FD02C02220CD
:1050600019F040E050E008C080910206482F552713
:10507000241735070CF4A9018091F905E82FFF27C3
:10508000FC83EB839F01E417F5070CF49A0120934E
:10509000C40229813A81261B370BB9016C0D7D1D95
:1050A00077FD02C0222019F080E090E007C08091D7
:1050B00002069927681779070CF4CB012B813C81F4
:1050C000281739070CF49C012093C5026091F5055F
:1050D0007091F60520913002309131024091C0026A
:1050E0005091C102241B350B621B730B882777FD7F
:1050F0008095982F0E94292E9B01AC01C301B2011B
:105100000E94502F0E940C2E7093C3026093C20223
:105110008091C2029091C3028C01222717FD209535
:10512000322F80915A0290915B02A0915C02B09163
:105130005D02080F191F2A1F3B1F00935A0210938C
:105140005B0220935C0230935D021016110612067A
:105150001306ACF4C80117FF03C0909581959F4FCB
:1051600060E071E00E94E72F6F5F7F4F882777FD37
:105170008095982F061B170B280B390B14C0C801FC
:1051800017FF03C0909581959F4F60E071E00E94EA
:10519000E72F6F5F7F4F882777FD8095982F060F49
:1051A000171F281F391F00935A0210935B02209388
:1051B0005C0230935D0280915A0290915B02A09153
:1051C0005C02B0915D0281383EE3930730E0A307B3
:1051D00030E0B3072CF080E89EE3A0E0B0E009C027
:1051E0008058914CAF4FBF4F64F480E891ECAFEF23
:1051F000BFEF80935A0290935B02A0935C02B0933E
:105200005D026091C2027091C302882777FD80958C
:10521000982F0E94292E7B018C0160915A02709177
:105220005B0280915C0290915D020E94292E9B019D
:10523000AC01C501B4010E94502F9B01AC01C80113
:10524000B7010E947E2D0E940C2E29813A81260FE3
:10525000371F2C193D0937FD02C0222019F040E00C
:1052600050E008C080910206482F552724173507C3
:105270000CF4A9012B813C81241735070CF49A0109
:105280002093EC0289819A81861B970BBC016C19D3
:105290007D0977FD02C0222019F020E030E008C02F
:1052A00080910206282F3327621773070CF49B01A5
:1052B0008B819C81821793070CF4C9018093D602DD
:1052C00024960FB6F894DEBF0FBECDBFDF91CF910D
:1052D0001F910F91FF90EF90DF90CF90BF90AF9014
:1052E0009F908F907F906F905F904F903F902F9006
:1052F00008952F923F924F925F926F927F928F927A
:105300009F92AF92BF92CF92DF92EF92FF920F9354
:105310001F93CF93DF93CDB7DEB764970FB6F894A2
:10532000DEBF0FBECDBF80917005882309F4BFC3D7
:105330008091BC029091BD0201969093BD02809332
:10534000BC028230910581F18330910524F40197EC
:1053500009F090C008C08330910509F446C0049755
:1053600009F088C063C08091580590915905A091BB
:105370005A05B0915B058093900290939102A0939F
:105380009202B093930280915C0590915D05A0918B
:105390005E05B0915F058093A0029093A102A09357
:1053A000A202B093A30266C080915805909159055E
:1053B000A0915A05B0915B05809394029093950259
:1053C000A0939602B093970280915C0590915D0541
:1053D000A0915E05B0915F058093A4029093A50211
:1053E000A093A602B093A70245C080915805909162
:1053F0005905A0915A05B0915B058093980290934E
:105400009902A0939A02B0939B0280915C059091BF
:105410005D05A0915E05B0915F058093A802909311
:10542000A902A093AA02B093AB0224C080915805B0
:1054300090915905A0915A05B0915B0580939C020B
:1054400090939D02A0939E02B0939F0280915C0571
:1054500090915D05A0915E05B0915F058093AC02CF
:105460009093AD02A093AE02B093AF021092BD0232
:105470001092BC0260919002709191028091920210
:10548000909193022091940230919502409196025E
:1054900050919702620F731F841F951F20919C02E9
:1054A00030919D0240919E0250919F02E09098029F
:1054B000F090990200919A0210919B022E0D3F1DCF
:1054C000401F511F620F731F841F951F24E030E09F
:1054D00040E050E00E941C30CA01B9010E94292E10
:1054E0000E94332E0E940C2E5B016C016093C80257
:1054F0007093C9028093CA029093CB026091A0027C
:105500007091A1028091A2029091A3022091A40225
:105510003091A5024091A6025091A702620F731F1D
:10552000841F951F2091AC023091AD024091AE02D4
:105530005091AF02E090A802F090A9020091AA0257
:105540001091AB022E0D3F1D401F511F620F731FA4
:10555000841F951F24E030E040E050E00E941C30A2
:10556000CA01B9010E94292E0E94332E0E940C2EDE
:105570007B018C016093F1027093F2028093F3023D
:105580009093F4028091D4029091D502019709F092
:105590008EC28091250290912602181619060CF0F1
:1055A00086C28091DC029091DD02892B51F18091BD
:1055B000580590915905A0915A05B0915B058093CB
:1055C000CC029093CD02A093CE02B093CF028091F3
:1055D0005C0590915D05A0915E05B0915F0580939B
:1055E000DE029093DF02A093E002B093E10282E337
:1055F00090E09093A8018093A7011092DD02109291
:10560000DC028091CC029091CD02A091CE02B091AB
:10561000CF028A199B09AC09BD09898B9A8BAB8B88
:10562000BC8B2091E6023091E702442737FD40957C
:10563000542FBC01CD010E94B42F5B016C0160931B
:105640006402709365028093660290936702809172
:10565000DE029091DF02A091E002B091E1028E198A
:105660009F09A00BB10B8D879E87AF87B88B2091C8
:10567000E6023091E702442737FD4095542FBC01E4
:10568000CD010E94B42F1B012C016093680270931E
:10569000690280936A0290936B02809164059091F5
:1056A0006505A0916605B091670589879A87AB87E4
:1056B000BC872091E8023091E902309521953F4F57
:1056C000442737FD4095542FBC01CD010E94B42FD3
:1056D0003B014C01609374027093750280937602D3
:1056E000909377028091680590916905A0916A0571
:1056F000B0916B058D839E83AF83B8872091E802BC
:105700003091E902309521953F4F442737FD409570
:10571000542FBC01CD010E94B42F69837A838B83FF
:105720009C83609378027093790280937A029093BD
:105730007B02E090E202F090E302A60CB71CC81CCA
:10574000D91CC601B5010E94292E0E94332E5B018F
:105750006C010027F7FC0095102FC801B7010E94CB
:10576000292E9B01AC01C601B5010E94C62D0E94E5
:105770000C2E4B017093BF026093BE02E090E202D8
:10578000F090E30289819A81AB81BC81280E391E99
:105790004A1E5B1EC201B1010E94292E0E94332EB7
:1057A0005B016C010027F7FC0095102FC801B701C1
:1057B0000E94292E9B01AC01C601B5010E94C62D95
:1057C0000E940C2E9B017093C1026093C0028091D5
:1057D000D2029091D302881599052CF48091D202BF
:1057E0009091D30211C08091D2029091D3029095F2
:1057F00081959F4F881699065CF48091D202909112
:10580000D302909581959F4F9093BF028093BE02E3
:105810008091D2029091D302821793072CF4809149
:10582000D2029091D30211C08091D2029091D30202
:10583000909581959F4F281739075CF48091D2028B
:105840009091D302909581959F4F9093C102809340
:10585000C00289899A89AB89BC8980937C02909324
:105860007D02A0937E02B0937F028D859E85AF85D9
:10587000B8898093800290938102A0938202B093B2
:1058800083028091C30583FFACC08091E4029091B4
:10589000E50220911D0230911E02820F931F90930A
:1058A0006302809362028091620290916302885643
:1058B000914054F080916202909163028856914029
:1058C0009093630280936202E0906202F090630220
:1058D0006091C0027091C102882777FD8095982F52
:1058E0000E94292E1B012C01A0906202B09063023D
:1058F0000027F7FC0095102FC801B7010E94292E40
:105900000E94982FA20191010E94502F3B014C014F
:10591000CC24B7FCC094DC2CC601B5010E94292E12
:105920000E94C02D7B018C016091BE027091BF026C
:10593000882777FD8095982F0E94292E9B01AC0126
:10594000C801B7010E94502F9B01AC01C401B301F3
:105950000E947E2D0E94332E0E940C2E5B017093BC
:10596000BF026093BE026091620270916302E09098
:105970006202F0906302882777FD8095982F0E943D
:10598000292E0E94C02DA20191010E94502F3B019F
:105990004C010027F7FC0095102FC801B7010E94A9
:1059A000292E0E94982F7B018C01CC24B7FCC09437
:1059B000DC2CC601B5010E94292E9B01AC01C80157
:1059C000B7010E94502F9B01AC01C401B3010E949A
:1059D0007D2D0E94332E0E940C2E7093C102609385
:1059E000C0028091BE029091BF021816190694F46D
:1059F00089859A85AB85BC854A97A105B10514F1C7
:105A000089899A89AB89BC898D599F4FAF4FBF4F08
:105A1000ACF418C0892BB1F089859A85AB85BC851B
:105A2000875E9F4FAF4FBF4F6CF489899A89AB89CE
:105A3000BC8984369105A105B10524F41092BF02FA
:105A40001092BE028091C0029091C10218161906F0
:105A500094F48D819E81AF81B8854A97A105B105E7
:105A600014F18D859E85AF85B8898D599F4FAF4FB5
:105A7000BF4FACF418C0892BB1F08D819E81AF81EE
:105A8000B885875E9F4FAF4FBF4F6CF48D859E8565
:105A9000AF85B88984369105A105B10524F410922B
:105AA000C1021092C0021092D5021092D4026496E4
:105AB0000FB6F894DEBF0FBECDBFDF91CF911F911F
:105AC0000F91FF90EF90DF90CF90BF90AF909F909D
:105AD0008F907F906F905F904F903F902F900895A0
:105AE000FC014150504030F001900616D1F731973B
:105AF000CF0108958827992708955058192E72D1FB
:105B000001D022C1BA176207730784079507B1F164
:105B100088F40EF410940B2EBA2FA02D062E622FAF
:105B2000202D072E732F302D082E842F402D092E67
:105B3000952F502DFF275523B9F0591B49F0573E9B
:105B400098F0469537952795A795F0405395C9F756
:105B500076F0BA0F621F731F841F30F48795779514
:105B60006795B795F040939517FA0F2E0895BF1BD0
:105B7000BB27BA0B620B730B840BF6CFDEF65EC14C
:105B800050E449EC3FE02BED87D0BBC02BD101D0D6
:105B9000DBC0552359F0992369F09F575F57951B38
:105BA00033F442F4903811F4915805C0E5C091588F
:105BB0009F3F09F443C1BB27112462177307840771
:105BC00030F4660F771F881FBB1F915098F311D0D8
:105BD0000F920FD00F920DD0A0E826173707480775
:105BE0001B0609F0A048BA2F602D7F918F910024E9
:105BF0000895A0E80024621773078407B10528F010
:105C0000621B730B840BB1090A2A660F771F881F6A
:105C1000BB1FA69581F7089597FBF0D09F3738F00A
:105C2000FEE9F91B982F872F762F6B2F05C003C134
:105C30009695879577956795F150D0F73EF49095B6
:105C40008095709561957F4F8F4F9F4F0895E89491
:105C500003C097FB0EF4F3DFB62F672F782F892F41
:105C60009EE9002471C0D8D09F3760F40EF0E3C0E5
:105C70009FEB80E877276627089586957795679547
:105C8000B11D93959639C8F32EF4BB2319F06F5FBD
:105C90007F4F8F4FBB2758C05F77552319F444239C
:105CA0000AF06AC02F933F934F935F936FDF55279E
:105CB0004427C6D05F914F913F912F91F1C00ED0F4
:105CC0005EF004C00BD026F001C008D019F020F41B
:105CD0008FEF089580E0089581E0089597FB092EE5
:105CE000052600F8689481D0E89407FC07C0621785
:105CF00073078407950721F008F40094079498949B
:105D000008951F939F7750EC49E43FE02BEDF6DEBA
:105D100010E89F775FE349EC3FE02BED62177307D4
:105D20008407950720F050EC49E4E8DE112713D1F1
:105D30009068E0E7F0E023D091271F9108959A95AD
:105D4000BB0F661F771F881F11249923A1F088239A
:105D5000B2F79F3F59F0BB0F48F421F4002011F433
:105D600060FF04C06F5F7F4F8F4F9F4F881F9795D5
:105D7000879597F908955FC09FEF80EC0895FF9293
:105D8000EF92DF92CF92BF926B017C01B59016D05B
:105D9000B590BB2069F09F938F937F936F93B6016B
:105DA000C7010CD02F913F914F915F910E94C62D5A
:105DB000BF90CF90DF90EF90FF900895D0D002C0B9
:105DC0009601A701EF93FF930E94502FFF91EF914F
:105DD000C6D0EF93FF930E947E2DFF91EF91BA946E
:105DE00079F70895052E092607FA440F551F5F3FDE
:105DF00079F0AA27A51708F051E04795880F991F59
:105E00009F3F31F0BB27B91708F091E087950895BF
:105E10009F919F911124B0CF97FB880F991F9F3FAF
:105E200031F0BB27B91708F091E0879508959F914D
:105E30009F911124A1CF6627772788279927089556
:105E4000EBDFCF93DF93D52FC42F5527442733277C
:105E500022279923D9F09F37C8F0F92F75DF592FE2
:105E6000482F372F262FF63968F4D6DEF2DEC03001
:105E7000CD0721F069937993899399939058DF9195
:105E8000CF913CCE9927882777276627C030CD074A
:105E900021F02993399349935993DF91CF9154CFAE
:105EA000A1DF01D051CF992339F0552329F09F5715
:105EB0005F57950F13F49AF1C1CF91589F3FE1F3CB
:105EC000629FA12D0F92BB27639FA00DB11DEE27EE
:105ED000729FA00DB11DEE1FAF93AA27649FB00D56
:105EE000E11D739FB00DE11DAA1F6627829FB00DB3
:105EF000E11DA61F5527749FE00DA11D551F839F0F
:105F0000E00DA11D561F849FA00D511D852F7A2FD6
:105F10006E2F1F900F9088231AF4939539F42CCF8D
:105F2000000C111CBB1F661F771F881F01280895D6
:105F30009F939F77993358F050E449EC3FE02BED65
:105F4000ABDE5FEB49EC3FE02BEDD8DDDADE5F91B5
:105F50005078952708959B01AC010C94502F5591D2
:105F60004591359125910895629FD001739FF0016D
:105F7000829FE00DF11D649FE00DF11D929FF00DD9
:105F8000839FF00D749FF00D659FF00D9927729F10
:105F9000B00DE11DF91F639FB00DE11DF91FBD019B
:105FA000CF0111240895AA1BBB1B51E107C0AA1FF2
:105FB000BB1FA617B70710F0A61BB70B881F991FAA
:105FC0005A95A9F780959095BC01CD01089597FB4E
:105FD000092E07260AD077FD04D0E5DF06D0002081
:105FE0001AF4709561957F4F0895F6F79095819515
:105FF0009F4F0895A1E21A2EAA1BBB1BFD010DC0E5
:10600000AA1FBB1FEE1FFF1FA217B307E407F50768
:1060100020F0A21BB30BE40BF50B661F771F881F44
:10602000991F1A9469F760957095809590959B01DA
:10603000AC01BD01CF01089597FB092E05260ED0B6
:1060400057FD04D0D7DF0AD0001C38F45095409596
:10605000309521953F4F4F4F5F4F0895F6F790953C
:106060008095709561957F4F8F4F9F4F0895F99957
:10607000FECFB2BDA1BDF89A119600B40895F9996A
:10608000FECFB2BDA1BD00BC11960FB6F894FA9A2E
:08609000F99A0FBE0895FFCF3D
:1060980001640A016400007D0000FF03010203049B
:1060A80005060708090A48616C6C6F2057656C740F
:1060B80000000000000000000000000000000000D8
:1060C80000000000000000000000000000000000C8
:1060D80000000000000000000000000000000000B8
:1060E80000000000000000000000000000000000A8
:1060F8000000000000000A014B616D65726100003C
:106108004E6F726D616C00000000803F17B7D13888
:0A61180030FB103A403296020A6490
:00000001FF
